:020000040000FA
:10000000D1EF03F01200FFFF04EF04F01200FFFF36
:10001000FFFFFFFFFFFFFFFF0CEF04F01200FFFFE9
:10002000FFFFFFFFFFFFFFFFFFFF0100CE07000004
:100030006A00000002000000126A1E0E716E0401C8
:10004000400E096F200E0A6F040E0B6F880E086FAA
:100050000401200E0E6F040E0F6F400E0C6F120085
:10006000550EA76EAA0EA76EA68212000401140EEA
:10007000226F010E236F1200106A04012151105CDF
:100080001CE2166A176A22511024F36E23511620BF
:10009000F46E24511720F86EF4CFF7FFF3CFF6FF7C
:1000A0000800F550116E1050EA6A250FE96E040E33
:1000B000EA2211C0EFFF102AE0D7F86A1200F00E12
:1000C00004012217840EA66E106A04012151105CEF
:1000D00023E21050EA6A250FE96E040EEA22EFCF00
:1000E00018F01050156E166A176A22511024F36E1C
:1000F00023511620F46E24511720F86EF4CFF7FF29
:10010000F3CFF6FF18C0F5FF0C000F0E10140F0808
:1001100001E1A6DF102AD9D71200940EA66E106A4C
:1001200004012151105C1DE21050156E166A060E76
:10013000D89015361636E804FBE1176A16BE176824
:10014000040122511524F36E23511620F46E24511C
:100150001720F86EF4CFF7FFF3CFF6FF81DF102AF8
:10016000DFD7F86A1200A66A106A04012151105CF8
:100170000EE222511024A96EA6801050EA6A250FC3
:10018000E96E040EEA22A8CFEFFF102AEED7120084
:10019000106A04012151105C12E222511024A96E50
:1001A0001050EA6A250FE96E040EEA22EF50A86E9D
:1001B000040EA66E55DFA6B2FED7102AEAD71200AB
:1001C000C40EA66E106A04012151105C1FE210508B
:1001D000EA6A250FE96E040EEA22EFCF18F01050FC
:1001E000156E166A176A22511024F36E23511620D9
:1001F000F46E24511720F86EF4CFF7FFF3CFF6FF1B
:1002000018C0F5FF0C002CDF102ADDD7F86A1200A9
:1002100079D8060E015C03E36D50020B01E071D04A
:10022000120410E104010CBF0CD00401400E096F50
:10023000400E040108170401087D880E040108130C
:10024000126A5FD0040108BF5CD0106A040120511B
:10025000320A3BE0CD0A2DE0F80A27E0020A21E04D
:10026000010A1BE0070A15E0010A0FE0030A09E092
:10027000070A07E0060A01E035D0F8DE040E106E2A
:1002800032D0FADE050E10262ED019DF010E106EC8
:100290002AD043DF010E106E26D065DF050E102632
:1002A00022D076DF010E106E1ED08ADF010E106E96
:1002B0001AD06D96136A146A1306000E145A13505E
:1002C000141001E0F9D7FF000ED0030E0401215DE8
:1002D00002E1010E106E040E0401215D02E1010E27
:1002E000106E01D000D0010E126E10500AE010C046
:1002F0000DF4400E04010C1704010C7D880E04015E
:100300000C13120000016A516B1104E1200E6A6F98
:100310004E0E6B6F6A07000E6B5B6DA208D06A51C0
:100320006B112DE18B708B50010B12E125D0015028
:1003300002E18B9021D0010402E18B8009D0020EF2
:10034000015C02E18B8018D0030E015C03E18B900D
:100350008B821200050E015C05E16A516B110FE101
:100360008B700AD0060E015C0AE16A516B1107E13D
:100370008B708B50010B02E08B9212008B8212006B
:100380006C500BE1040100513C0BE842E8420D08BF
:1003900002E1D2EF01F0DAEF01F0040E6C5C01E152
:1003A00017D81200056A066A0B6A0C6AFBEC02F0A9
:1003B00058EF02F0020E055C09E157D8040100BDB8
:1003C00002D0C80E01D0880E006F120096EF02F026
:1003D000040E015C09E112C46EFF6E50000802E2D7
:1003E000050E01D0030E016E050409E10AD80401CF
:1003F00004BD02D0C80E01D0880E046F120096EF23
:1004000002F0080E0B5C000E0C5802E20B5001D0FB
:10041000080E0E6EE8CF05F4166AE8500B5E165013
:100420000C5A180E096E040E0A6E0E501DE002A240
:1004300007D007C0F6FF08C0F7FF0800F55005D049
:1004400007C0E9FF08C0EAFFEF50E66E09C0E9FF08
:100450000AC0EAFFE552E750EF6E072A000E0822B5
:10046000092A0A220E06E1D7120001C40FF00F502C
:100470000B240B6E000E0C200C6E180E076E040E73
:10048000086E0F5014E007C0E9FF08C0EAFFEF5004
:10049000E66E09C0E9FF0AC0EAFFE552E750EF6ED9
:1004A000092A000E0A22072A08220F06EAD712009C
:1004B0006D9806500BE10401080E016F100E026FDB
:1004C000040E036F840E006F04011ED0040110AFF0
:1004D0001DD00B50165D0C50175904E216C40BF0DA
:1004E00017C40CF08EDF010E056E0401080E016FBB
:1004F000100E026F040E036F800E006F0401180EC1
:10050000066F040E076FC80E046F1200020E056E10
:100510000401056BC80E046F0401080E016F180E6C
:10052000026F040E036FC80E006F1200056A04010B
:10053000080E016F100E026F040E036F8C0E006F19
:100540000401046B1200080E6D6E6DBAFED7686A66
:10055000110E696E020E016E12006850040B09E064
:100560006950040B06E06D92699468A402D0689407
:10057000FCD76850010B04E06950010B01E024D85E
:100580006850100B0AE06950100B07E06984689806
:100590006D82A19AA08A0300A19A6850200B06E000
:1005A0006950200B03E070B07090689A030E015CF4
:1005B00001E209D06850080B06E06950080B03E01F
:1005C000C0EC01F068961200686A7B0E696E6E6A74
:1005D000160E706E68A608D0689600000000000035
:1005E000000000000000F6D76D9896EC02F0036A58
:1005F000030E016E120004011051600BE842E84244
:10060000E842E842E842000901E012001151080AFC
:100610002FE0010A2BE00F0A08E0030A01E01200B4
:10062000010E066E040E016E1200010E066E130519
:1006300006E13E0E076E070E086E120E11D0020E76
:10064000135D06E1500E076E070E086E200E08D0EF
:10065000030E135D08E1700E076E070E086E040EA0
:100660000B6E0C6A01D0066A0282120042EF03F0A0
:10067000010E066E030E076E000E086E0292010E4A
:100680000B6E1200010E066E12C403F0040112512B
:1006900003E1050E016E1200060E016E1CEF00F064
:1006A0002A0EF66E000EF76E000EF86E00010900BD
:1006B000F550656F0900F550666F03E1656701D07D
:1006C0003DD00900F550606F0900F550616F0900D9
:1006D000F550626F09000900F550E96E0900F55008
:1006E000EA6E090009000900F550636F0900F55032
:1006F000646F09000900F6CF67F0F7CF68F0F8CF14
:1007000069F060C0F6FF61C0F7FF62C0F8FF00014A
:10071000635302E1645307E00900F550EE6E63078E
:10072000F8E26407F9D767C0F6FF68C0F7FF69C051
:10073000F8FF00016507000E665BBFD712001201CB
:10074000000200000008D8040B00010000000001B6
:1007500009022000010100803209040000020000AB
:10076000000007050102400000070581024000006B
:1007700004030904C150006E0F0EC11282A404D0FC
:100780000050C16E00EF04F08B6AFC0E946E140EE4
:100790006F6EA3EC02F0ADEC02F008EC01F0FBD7B9
:1007A000120013EE00F023EE00F0F86A1A9C50ECF1
:1007B00003F0E6EC03F0BAEC03F0FBD7120000EE16
:1007C00000F00F0EEE6AEA62FDD712001200000080
:1007D000FFFFFFFFFFFFFFFFFFFFFFFFFFFFFFFF29
:1007E000FFFFFFFFFFFFFFFFFFFFFFFFFFFFFFFF19
:1007F000FFFFFFFFFFFFFFFFFFFFFFFFFFFFFFFF09
:10080000DDEF22F01200FFFFBBEF05F01200FFFF4B
:10081000FFFFFFFFFFFFFFFF22EF04F01200FFFFCB
:10082000FFFFFFFFFFFFFFFFFFFF02000C4600007E
:10083000DC0100000200000008460000D6010000B4
:1008400004000000D8CFE4FFE0CFE4FFE46EDACF8D
:10085000E4FFE2CFDAFFE9CFE4FFEACFE4FFF3CF32
:10086000E4FFF4CFE4FFE6529EA201D19E92030E74
:10087000386E0E50EA6A510FE96E010EEA22EF500F
:10088000385C30E10E50E96EEA6AD890E936EA3613
:10089000690EE926010EEA22EECF38F0EFCF39F0EB
:1008A00039C038F0396A3850D76E0E50E96EEA6AAE
:1008B000D890E936EA36690EE926010EEA22EECF33
:1008C00038F0EFCF39F03850D66EF28AF294D58EE8
:1008D0000E50EA6A510FE96E010EEA22040EEF6E25
:1008E0000E50106E020E386E0F50EA6A510FE96E0C
:1008F000010EEA22EF50385C49E10F50E96EEA6AD6
:10090000D890E936EA36690EE926010EEA22EE5061
:10091000ED1009E10F50EA6A510FE96E010EEA226B
:10092000010EEF6E33D0080E0F5C0CE2070E0F14B1
:10093000386E010E385204E0E846FE0B3806FCE142
:1009400089121AD0100E0F5C0CE2070E0F14386ECD
:10095000010E385204E0E846FE0B3806FCE18A122C
:100960000BD0070E0F14386E010E385204E0E84623
:10097000FE0B3806FCE18B120F50EA6A510FE96E4C
:10098000010EEA22030EEF6E0F500E6E0F2A060EB6
:100990000F5C03E1080E0F6E0AD0130E0F5C03E12B
:1009A000160E0F6E04D0180E0F5C01E10F6A000ED8
:1009B000D8800254000E03542EE2112A000E122297
:1009C0000250115C0350125826E3116A126A030E9A
:1009D000065C1FE20450EA6A480FE96E010EEA2243
:1009E00080CFEFFF0450EA6A4B0FE96E010EEA2256
:1009F00081CFEFFF0450EA6A4E0FE96E010EEA2242
:100A000082CFEFFF042A030E045C01E3046A062A86
:100A100002D0026A036A000ED8800754000E085400
:100A200019E20C50000816E2132A000E1422075097
:100A3000135C085014580EE3136A146A030E0B5C1F
:100A400007E2092A030E095C01E3096A0B2A02D0B6
:100A5000076A086A0C5000080AE2156A1550040D6E
:100A6000F328C26E9E9C9F9C9D8CC280C2829EACCD
:100A70002DD09E9CC4503C6E3CC03DF03C6AC3509F
:100A800000013C103A6E3DC03BF01550060DF3CF0F
:100A900038F0F4CF39F0000E3826010E3922095013
:100AA000020D3850F324E96E3950F420EA6E3AC052
:100AB000EEFF3BC0EDFF152A0C50155C02E39D9C38
:100AC00005D01550040DF328C26EC282F2A442D0A4
:100AD000D59EF294F29A040E386E1050EA6A510FC5
:100AE000E96E010EEA22EF50385C34E1080E105C2A
:100AF0000DE2070E1014386E010E385204E0E8467D
:100B0000FE0B3806FCE1E81C89161CD0100E105CA8
:100B10000DE2070E1014386E010E385204E0E8465C
:100B2000FE0B3806FCE1E81C8A160CD0070E1014E8
:100B3000386E010E385204E0E846FE0B3806FCE140
:100B4000E81C8B161050EA6A510FE96E010EEA227A
:100B5000020EEF6EE552E5CFF4FFE5CFF3FFE5CFF0
:100B6000EAFFE5CFE9FFE5CFDAFFE550E5CFE0FFAB
:100B7000E5CFD8FF1000DACFE4FFE2CFDAFFE6528C
:100B8000E552E5CFDAFF1100D9CFE6FFE1CFD9FF7B
:100B9000020EE126896A92680F0EC16EC2900C6A3D
:100BA000070EB46E8A6A93688B6A9468FC0E8B1683
:100BB000FC0E941694840101010EBE6F0101DC69E4
:100BC000DD690A6A096A0B6A056A046A066A026ACA
:100BD000036A076A086A116A126A136A146A156A54
:100BE000CA82CA80CA9CCA9ACA88CA96FA0ECB6EB2
:100BF000DF6ADFCF2AF00C0EE76E2A18E8AE02D0CB
:100C0000E73402D0E7502A5C38E2010EDB6A010EBD
:100C1000DBCF2AF0030EE76E2A18E8AE02D0E734E5
:100C200002D0E7502A5C27E2DFCF2AF02B6A2ABEE7
:100C30002B68060E2B02F3CF2BF0060E2A02F3CF01
:100C40002AF0F4502B26000E2A26010E2B22010E2C
:100C5000DBCF2CF02D6A2CBE2D68D8902C362D368B
:100C60002A502C24E96E2B502D20EA6EEE6AED6A94
:100C7000010EDB2ACCD7DF2ABCD70101B86B0101FA
:100C8000B96B0101B66B0101B76B0101BA6B0101D0
:100C9000BB6B0101BC6B0101BD6B0E6A0F6A106A70
:100CA000DF6ADFCF2AF0180EE76E2A18E8AE02D00E
:100CB000E73402D0E7502A5C1BE2DFCFE9FFEA6AA3
:100CC000E9BEEA68D890E936EA36690EE926010EEF
:100CD000EA22EE6AED6ADFCFE9FFEA6AE9BEEA6876
:100CE000510EE926010EEA22010EEF6EDF2AD9D756
:100CF000D586D59AD59CF294F29AF194D08ECA9466
:100D00009D829F92F28EF28CCA84020EE15C02E216
:100D1000E16AE552E16EE552E7CFD9FF1200D9CF83
:100D2000E6FFE1CFD9FF020EE126010EDB6A0101E9
:100D3000996B11EC13F00650000809E20AEC0BF075
:100D4000052A030E055C01E1056A0606F4D70B507F
:100D5000000809E236EC0BF00A2A030E0A5C01E1F6
:100D60000A6A0B06F4D7040104011851800B6CE1E8
:100D7000060E0101D25D68E36D50020B65E10101D1
:100D8000996B040119510101995D53E201019951D7
:100D9000EA6A080FE96E050EEA22EFCFDFFF0101D4
:100DA000D6511CE10D0E2A6EDF502A5C05E00A0EBA
:100DB0002B6EDF502B5C12E10101010ED66F010199
:100DC000B851EA6A400FE96E020EEA220D0EEF6E8C
:100DD0000101B82BDE52010EDD6E15D00D0EDF5C69
:100DE00011E00A0EDF5C0EE00101B851EA6A400F23
:100DF000E96E020EEA22DFCFEFFF0101D66B01019F
:100E0000B82B01D013D0400E0101B85D02E1010101
:100E1000B86B0101B9510101B85D02E10D8609D03D
:100E2000010EDB5003E01CD9010EDB6A0101992B96
:100E3000A8D70401400E196F400E040118170401D1
:100E4000187D880E040118130D5001E181D00DA00A
:100E500010D05F0E2A6E400E2B6E2C6A2AC0E6FF61
:100E60002BC0E6FF2CC0E6FF5FEC21F0E552E55217
:100E7000E5520DA210D0590E2A6E400E2B6E2C6A30
:100E80002AC0E6FF2BC0E6FF2CC0E6FF5FEC21F096
:100E9000E552E552E5520DA410D03D0E2A6E400EEB
:100EA0002B6E2C6A2AC0E6FF2BC0E6FF2CC0E6FFA3
:100EB0005FEC21F0E552E552E5520DA610D0210E6F
:100EC0002A6E400E2B6E2C6A2AC0E6FF2BC0E6FF6E
:100ED0002CC0E6FF5FEC21F0E552E552E5520DA88B
:100EE00010D0020E2A6E400E2B6E2C6A2AC0E6FF2E
:100EF0002BC0E6FF2CC0E6FF5FEC21F0E552E55287
:100F0000E5520DAA00D00DAC10D0E10E2A6E3F0EB6
:100F10002B6E2C6A2AC0E6FF2BC0E6FF2CC0E6FF32
:100F20005FEC21F0E552E552E5520DAE10D0C80E4F
:100F30002A6E3F0E2B6E2C6A2AC0E6FF2BC0E6FFFE
:100F40002CC0E6FF5FEC21F0E552E552E5520D6A58
:100F500035D8020EE15C02E2E16AE552E16EE5524B
:100F6000E7CFD9FF1200D9CFE6FFE1CFD9FF0101CA
:100F7000B651EA6A000FE96E020EEA22FE0EDBCFDE
:100F8000EFFF0101B62B400E0101B65D02E1010148
:100F9000B66B0101B7510101B65D01E10D84FE0E92
:100FA000DBCF2AF02B6A2ABE2B682AC0F3FF2BC0A6
:100FB000F4FF00D0E552E7CFD9FF1200D9CFE6FF0A
:100FC000E1CFD9FFE65201019A5145E1060E010138
:100FD000D25D41E36D50020B3EE10101B6510101CA
:100FE000B75D39E00101B7510101D880B6551AE269
:100FF0000101B7510101B65DDF6E0101B751010179
:101000009B6F9C6B000E01019B27020E01019C232C
:10101000DFCF9FF10101A06B0101010E9A6FB6C1F4
:10102000B7F119D0400E0101D880B755DF6E01012C
:10103000B75101019B6F9C6B000E01019B27020EB3
:1010400001019C23DFCF9FF10101A06B0101010E83
:101050009A6F0101B76BE552E552E7CFD9FF120055
:10106000D9CFE6FFE1CFD9FF040EE126DE6ADD6AC3
:10107000020EDB6A030EDB6A0101B951EA6A400F16
:10108000E96E020EEA22EF50E66EE66A58EC22F0B4
:10109000E552E552020EF3CFDBFF0101B92B400E02
:1010A0000101B95D02E10101B96B020EDB50DE6E98
:1010B000DD6A0101B951EA6A400FE96E020EEA22C7
:1010C000EF502C0835E00101B951EA6A400FE96E92
:1010D000020EEA22EF500D082BE00101B951EA6A35
:1010E000400FE96E020EEA22EF50E66EE66A58EC17
:1010F00022F0E552E552030EF3CFDBFF0101B92BDD
:10110000400E0101B95D02E10101B96B020EDBCFB6
:101110002CF02CC02DF02C6A030EDB5000012C2487
:101120002A6E000E2D202B6E2AC0DEFF2BC0DDFFA5
:10113000000EDBCF1EF0010EDBCF1FF0490E1E1894
:1011400002E1430E1F1801E1D7D0490E1E1802E13B
:10115000520E1F1801E1CDD0490E1E1802E1530EA8
:101160001F1801E1C3D0530E1E1802E1430E1F18D1
:1011700001E1B9D0530E1E1802E1520E1F1801E111
:10118000AFD0530E1E1802E1530E1F1801E1A5D077
:10119000530E1E1802E1420E1F1801E19BD0430EB0
:1011A0001E1802E1420E1F1801E191D0430E1E18D5
:1011B00002E1520E1F1801E187D04F0E1E1802E106
:1011C000420E1F1801E17DD0570E1E1802E14D0E90
:1011D0001F1875E0520E1E1802E14D0E1F186DE02B
:1011E000440E1E1802E1500E1F1865E04F0E1E1827
:1011F00002E1500E1F185DE0490E1E1802E1500E6C
:101200001F1855E0580E1E1802E1540E1F184CE02E
:10121000540E1E1801E11F5045E0410E1E1801E159
:101220001F503EE0560E1E1801E11F5037E0490ED8
:101230001E1801E11F5030E04F0E1E1801E11F5033
:1012400029E0550E1E1802E1430E1F1821E0580E2A
:101250001E1802E1430E1F1818E0430E1E1801E18C
:101260001F5011E0520E1E1801E11F500AE0580EE7
:101270001E1802E1520E1F1801E041D0C4EC0DF01F
:101280007DD0B3D87BD036D979D0C6EC0DF076D0EE
:10129000B0D874D08CD972D0BDD970D0D6D96ED018
:1012A000E5D96CD0E6D86AD0C2EC0DF067D051DB3E
:1012B00065D0CFDB63D0B1DA61D06EDA5FD037DAD8
:1012C0005DD0B4EC0EF05AD0C8EC0DF057D06DECF8
:1012D0000EF054D0FBEC0FF051D0B7EC10F04ED024
:1012E000BAEC10F04BD0BDEC10F048D0C0EC10F0D0
:1012F00045D0C3EC10F042D0C6EC10F03FD0030E46
:10130000DB501AE1020EDBCFE6FFE66A020EDBCF0E
:10131000E6FFE66AA50E2A6E3F0E2B6E2C6A2AC0E7
:10132000E6FF2BC0E6FF2CC0E6FF5FEC21F02D6E40
:10133000070EE15E2D5021D0030EDBCFE6FFE66AFB
:10134000020EDBCFE6FFE66A030EDBCFE6FFE66ABE
:10135000020EDBCFE6FFE66A7D0E2A6E3F0E2B6E95
:101360002C6A2AC0E6FF2BC0E6FF2CC0E6FF5FEC2C
:1013700021F02D6E0B0EE15E2D5000D00101B95110
:10138000EA6A400FE96E020EEA22EF500D080DE006
:101390000D500BE1520E2A6E2B6ADF502A1803E122
:1013A000DE52DD502B1801E00D8EB8C1B9F1040EEC
:1013B000E15C02E2E16AE552E16EE552E7CFD9FF76
:1013C00012000101BE5110E07C0E2A6E450E2B6EFC
:1013D0002C6A2AC0E6FF2BC0E6FF2CC0E6FF5FECBC
:1013E00021F0E552E552E5521200C4EC05F0E9DFC8
:1013F0001200D9CFE6FFE1CFD9FF030EE126010E9F
:10140000E66EC9EC10F0E5521D50DF6E020EE66E7E
:10141000C9EC10F0E552DE521DC0DEFF1EC0DDFF3C
:10142000DD520D5001E01BD0DF0418E1D950010F4F
:10143000E96EDACFEAFFEE50ED100BE0010E2A6EF6
:101440002B6A010EDB502A1803E1020EDB502B1829
:1014500004E1010EDBCFBEF101D00D8CB2DF030E33
:10146000E15C02E2E16AE552E16EE552E7CFD9FFC5
:101470001200D9CFE6FFE1CFD9FF030EE126020E1D
:10148000DB6A030EE66EC9EC10F0E5521DC000F0F9
:101490001EC001F0010EE66EC9EC10F0E552020E1E
:1014A0001DC0DBFF0D5001E01BD0020EDB500CE134
:1014B0000050011003E1026A036A05D0CA8400C02B
:1014C00002F001C003F00BD00050011003E1076AE5
:1014D000086A05D0CA8400C007F001C008F071DFB7
:1014E000030EE15C02E2E16AE552E16EE552E7CF0C
:1014F000D9FF1200D9CFE6FFE1CFD9FF040EE126D4
:10150000010EE66EC9EC10F0E5521D50DF6E010EC3
:10151000E66EC9EC10F0E552010E1DC0DBFF010EB6
:10152000E66EC9EC10F0E552020E1DC0DBFF010EA5
:10153000E66EC9EC10F0E552030E1DC0DBFF0D5046
:1015400001E02BD0DF50926E010EDB50936E020E45
:10155000DB50946E030EDB500C0805E20C0EF36EAC
:10156000030EF3CFDBFF030EDB5005E10F0EC16E60
:10157000C2900C6A11D00C6AC26A030EDBCFE6FF80
:101580000F0EE552D880E754C16EBE0EC06EC28009
:10159000030EDB500C6ECA8414DF040EE15C02E221
:1015A000E16AE552E16EE552E7CFD9FF1200D9CFEB
:1015B000E6FFE1CFD9FF030EE126010EE66EC9EC8E
:1015C00010F0E5521D50DF6E010EE66EC9EC10F012
:1015D000E552010E1DC0DBFF010EE66EC9EC10F0F6
:1015E000E552020E1DC0DBFF0D5001E009D0DF50B7
:1015F000896E010EDB508A6E020EDB508B6EE1DECF
:10160000030EE15C02E2E16AE552E16EE552E7CFEA
:10161000D9FF12008250E66EE66A8150E66EE66AF5
:101620008050E66EE66A6A0E2A6E3F0E2B6E2C6ABA
:101630002AC0E6FF2BC0E6FF2CC0E6FF5FEC21F0DE
:101640002D6E090EE15E2D501200840E2A6E450E9D
:101650002B6E2C6A2AC0E6FF2BC0E6FF2CC0E6FFEB
:101660005FEC21F0E552E552E5521200D9CFE6FFDA
:10167000E1CFD9FFE652DF6A680E2A6E3F0E2B6E6D
:101680002C6A2AC0E6FF2BC0E6FF2CC0E6FF5FEC09
:1016900021F0E552E552E552DF6A0C50DF5C32E2A0
:1016A000DFCF2AF02B6A2ABE2B68060E2B02F3CF5F
:1016B0002BF0060E2A02F3CF2AF0F4502B26000E50
:1016C0002A26010E2B220A50020D2A50F324E96E1D
:1016D0002B50F420EA6EEECFE6FFEFCFE6FF620E6E
:1016E0002C6E3F0E2D6E2E6A2CC0E6FF2DC0E6FF3D
:1016F0002EC0E6FF5FEC21F02F6E050EE15E2F504D
:10170000DF2ACBD7810E2A6E450E2B6E2C6A2AC09B
:10171000E6FF2BC0E6FF2CC0E6FF5FEC21F0E552B0
:10172000E552E552E552E552E7CFD9FF1200D9CF95
:10173000E6FFE1CFD9FF030EE126030EE66EC9EC0A
:1017400010F0E5521DC0DEFF1EC0DDFF010EE66E8B
:10175000C9EC10F0E552020E1DC0DBFF0D5001E098
:1017600011D0DECF2AF0DDCF2BF0000E2A5C100E58
:101770002B5807E2DECFE9FFDDCFEAFF020EDBCF19
:10178000EFFF1FDE030EE15C02E2E16AE552E16E6B
:10179000E552E7CFD9FF1200D9CFE6FFE1CFD9FF5D
:1017A000030EE126030EE66EC9EC10F0E5521DC0F3
:1017B000DEFF1EC0DDFF0D5001E025D0DECF2AF098
:1017C000DDCF2BF0000E2A5C100E2B5807E2DECF87
:1017D000E9FFDDCFEAFF020EEFCFDBFF020EDBCF2A
:1017E000E6FFE66A580E2A6E3F0E2B6E2C6A2AC060
:1017F000E6FF2BC0E6FF2CC0E6FF5FEC21F02D6E6C
:10180000050EE15E2D50030EE15C02E2E16AE55255
:10181000E16EE552E7CFD9FF1200D9CFE6FFE1CF65
:10182000D9FF030EE126050EE66EC9EC10F0E55275
:101830001D50DF6E010EE66EC9EC10F0E552010E90
:101840001DC0DBFF010EE66EC9EC10F0E552020E82
:101850001DC0DBFF0D5001E072D0020EDB5001080D
:1018600002E20D8C6CD0010EDB50070802E20D8CF9
:1018700066D0410E2A6EDF502A5C1CE1020EDB505E
:101880000DE1010EF36E010EDB5004E0D890F3364B
:10189000E806FCE1F350E81C92160BD0010EF36E43
:1018A000010EDB5004E0D890F336E806FCE1F3507B
:1018B000921244D0420E2A6EDF502A5C1CE1020EC6
:1018C000DB500DE1010EF36E010EDB5004E0D89009
:1018D000F336E806FCE1F350E81C93160BD0010E3A
:1018E000F36E010EDB5004E0D890F336E806FCE11D
:1018F000F350931223D0430E2A6EDF502A5C1CE172
:10190000020EDB500DE1010EF36E010EDB5004E020
:10191000D890F336E806FCE1F350E81C94160BD09F
:10192000010EF36E010EDB5004E0D890F336E806AA
:10193000FCE1F350941202D00D8C01D042DD030E75
:10194000E15C02E2E16AE552E16EE552E7CFD9FFE0
:101950001200D9CFE6FFE1CFD9FF030EE126020E38
:10196000DB6A050EE66EC9EC10F0E5521D50DF6E25
:10197000010EE66EC9EC10F0E552010E1DC0DBFF52
:101980000D5001E05CD0010EDB50070802E20D8C27
:1019900056D0410E2A6EDF502A5C10E1010EF36E24
:1019A000010EDB5004E0D890F336E806FCE1F3507A
:1019B0008014E76E020EE7CFDBFF2CD0420E2A6EBA
:1019C000DF502A5C10E1010EF36E010EDB5004E0E3
:1019D000D890F336E806FCE1F3508114E76E020E6E
:1019E000E7CFDBFF17D0430E2A6EDF502A5C10E1F1
:1019F000010EF36E010EDB5004E0D890F336E806DA
:101A0000FCE1F3508214E76E020EE7CFDBFF02D059
:101A10000D8C15D0020EDBCFE6FFE66A4F0E2A6E64
:101A20003F0E2B6E2C6A2AC0E6FF2BC0E6FF2CC0AF
:101A3000E6FF5FEC21F02D6E050EE15E2D50030EEA
:101A4000E15C02E2E16AE552E16EE552E7CFD9FFDF
:101A50001200D9CFE6FFE1CFD9FF030EE126050E34
:101A6000E66E97DBE5521D50DF6E010EE66E91DBF0
:101A7000E552010E1DC0DBFF010EE66E8ADBE5526A
:101A8000020E1DC0DBFF0D5001E072D0020EDB50D4
:101A9000010802E20D8C6CD0010EDB50070802E257
:101AA0000D8C66D0410E2A6EDF502A5C1CE1020EBE
:101AB000DB500DE1010EF36E010EDB5004E0D89017
:101AC000F336E806FCE1F350E81C89160BD0010E52
:101AD000F36E010EDB5004E0D890F336E806FCE12B
:101AE000F350891244D0420E2A6EDF502A5C1CE16A
:101AF000020EDB500DE1010EF36E010EDB5004E02F
:101B0000D890F336E806FCE1F350E81C8A160BD0B7
:101B1000010EF36E010EDB5004E0D890F336E806B8
:101B2000FCE1F3508A1223D0430E2A6EDF502A5C68
:101B30001CE1020EDB500DE1010EF36E010EDB50D5
:101B400004E0D890F336E806FCE1F350E81C8B166D
:101B50000BD0010EF36E010EDB5004E0D890F3368B
:101B6000E806FCE1F3508B1202D00D8C01D029DC89
:101B7000030EE15C02E2E16AE552E16EE552E7CF75
:101B8000D9FF12001EDC12001CDC12001ADC12004D
:101B9000D9CFE6FFE1CFD9FF040EE126050EE66EB0
:101BA000F8DAE5521D50DF6E010EE66EF2DAE5520C
:101BB000010E1DC0DBFF030EE66EEBDAE552020EEE
:101BC0001DC0DBFF030E1EC0DBFF0D5001E07BD00C
:101BD000D950020FE96EDACFEAFF720ED880EE54C8
:101BE0002E0EED5402E20D8C6ED0D950020FE96E2C
:101BF000DACFEAFFEE50ED101FE02D682E682F6A55
:101C00002D0EE76E020EDBCF30F0030EDBCF31F08E
:101C1000E7503026000E3122326A30502D5C2A6E99
:101C200031502E582B6E32502F582C6E020E2AC077
:101C3000DBFF030E2BC0DBFF010EDB50070802E2C7
:101C40000D8C41D0410E2A6EDF502A5C02E1DF6A22
:101C500012D0420E2A6EDF502A5C03E1080EDF6EBE
:101C60000AD0430E2A6EDF502A5C03E1100EDF6EAD
:101C700002D00D8C28D0010EDB50DF24E96EEA6A19
:101C8000D890E936EA36690EE926010EEA22020EFC
:101C9000DBCFEEFF030EDBCFEDFF010EDB50DF24C9
:101CA000EA6A510FE96E010EEA22EF040AE1010E21
:101CB000DB50DF24EA6A510FE96E010EEA22020EC0
:101CC000EF6EE1EC09F0040EE15C02E2E16AE5523C
:101CD000E16EE552E7CFD9FF1200D9CFE6FFE1CFA1
:101CE000D9FF050EE126010EE66E53DAE5521D50CE
:101CF000DF6E010EE66E4DDAE552020E1DC0DBFF0F
:101D0000010EE66E46DAE552030E1DC0DBFF010E42
:101D1000E66E3FDAE552010E1DC0DBFF010EE66EF6
:101D200038DAE552040E1DC0DBFF0D5001E012D081
:101D3000DFCFB1F1020EDBCFB3F1010EDBCFB2F199
:101D4000030EDBCFB4F1040EDBCFB5F1B1C189FFD7
:101D5000E1EC09F0050EE15C02E2E16AE552E16EB8
:101D6000E552E7CFD9FF1200D9CFE6FFE1CFD9FF87
:101D7000040EE126030EDB6A0101B951EA6A400F45
:101D8000E96E020EEA22EF502C081DE00101B95164
:101D9000EA6A400FE96E020EEA22EF50E66EE66A4A
:101DA000280E2A6E3F0E2B6E2C6A2AC0E6FF2BC02F
:101DB000E6FF2CC0E6FF5FEC21F02D6E050EE15E24
:101DC0002D500D8A0ED10101B92B400E0101B95DD4
:101DD00002E10101B96BB1C189FF0101B21D891492
:101DE0002A6E891C0101B2152A10E76E010EE7CF99
:101DF000DBFF0101B951EA6A400FE96E020EEA22E7
:101E0000EF500D0801E1EBD00101B951EA6A400F32
:101E1000E96E020EEA22EF50E66EE66A58EC22F016
:101E2000E552E552020EF3CFDBFF300EF36E020EE9
:101E3000DBCFF4FFF350F45C0FE3020EDB50390804
:101E40000BE3300E2A6E020EDBCFE7FF2A50E75E6F
:101E5000020EE7CFDBFF19D0410EF36E020EDBCF8F
:101E6000F4FFF350F45C0FE3020EDB5046080BE383
:101E7000370E2A6E020EDBCFE7FF2A50E75E020E16
:101E8000E7CFDBFF02D00D8CACD0020EDB38F00BBD
:101E9000DF6E0101B92B400E0101B95D02E10101C4
:101EA000B96B0D0E2A6E0101B951EA6A400FE96E55
:101EB000020EEA22EF502A5C02E10D8892D0010165
:101EC000B951EA6A400FE96E020EEA22EF50E66E5F
:101ED000E66A58EC22F0E552E552020EF3CFDBFF42
:101EE000300EF36E020EDBCFF4FFF350F45C0FE321
:101EF000020EDB5039080BE3300E2A6E020EDBCFE8
:101F0000E7FF2A50E75E020EE7CFDBFF19D0410E54
:101F1000F36E020EDBCFF4FFF350F45C0FE3020E1E
:101F2000DB5046080BE3370E2A6E020EDBCFE7FFCD
:101F30002A50E75E020EE7CFDBFF02D00D8C51D0B6
:101F4000020EDB50DF24DF6E0101B92B400E0101D0
:101F5000B95D02E10101B96BDF508A6E010EDB5001
:101F6000896E0101B55105E0B5C1E6FFE9EC22F04B
:101F7000E552B1C189FF0101B45130E0030EB4C193
:101F8000DBFF0101B1510101B3152A6E0101B3510B
:101F900080142A5C0BE1030EDB5008E00000000017
:101FA000000000000000030EDB06EBD7030EB4C1F7
:101FB000DBFF0101B1510101B3152A6E0101B351DB
:101FC00080142A5C0BE0030EDB5008E000000000E8
:101FD000000000000000030EDB06EBD70AD7E1EC9F
:101FE00009F0040EE15C02E2E16AE552E16EE552BD
:101FF000E7CFD9FF1200D9CFE6FFE1CFD9FF050E19
:10200000E126030EDB6A040EDB6A010EE66EC1D820
:10201000E552040E1DC0DBFF040EDB5004E0040E8D
:10202000DB50380802E20D8C98D00101B951EA6A00
:10203000400FE96E020EEA22EF502C081DE001016C
:10204000B951EA6A400FE96E020EEA22EF50E66EDD
:10205000E66A280E2A6E3F0E2B6E2C6A2AC0E6FF17
:102060002BC0E6FF2CC0E6FF5FEC21F02D6E050EC5
:10207000E15E2D500D8A71D00101B92B400E010196
:10208000B95D02E10101B96BB1C189FF0101B21D66
:1020900089142A6E891C0101B2152A10E76E010EFF
:1020A000E7CFDBFF040EDB5056E00101B951EA6ACD
:1020B000400FE96E020EEA22EFCFDFFF0101B92BDC
:1020C000400E0101B95D02E10101B96B040EDB06AE
:1020D000DF508A6E010EDB50896E0101B55105E0BB
:1020E000B5C1E6FFE9EC22F0E552B1C189FF01017B
:1020F000B45130E0030EB4C1DBFF0101B151010165
:10210000B3152A6E0101B35180142A5C0BE1030E52
:10211000DB5008E000000000000000000000030E9B
:10212000DB06EBD7030EB4C1DBFF0101B1510101A6
:10213000B3152A6E0101B35180142A5C0BE0030E23
:10214000DB5008E000000000000000000000030E6B
:10215000DB06EBD7A7D7E1EC09F0050EE15C02E264
:10216000E16AE552E16EE552E7CFD9FF1200E1ECFA
:1021700009F01200E1EC09F01200E1EC09F01200A4
:10218000E1EC09F01200E1EC09F01200E1EC09F0D9
:102190001200D9CFE6FFE1CFD9FF040EE126030EEE
:1021A000DB6A0D0E2A6E0101B951EA6A400FE96E31
:1021B000020EEA22EF502A5C05E10D881D6A1E6AB4
:1021C0001F6A93D10101B951EA6A400FE96E020E0C
:1021D000EA22EF502C0820E00101B951EA6A400FD1
:1021E000E96E020EEA22EF50E66EE66A280E2A6ECB
:1021F0003F0E2B6E2C6A2AC0E6FF2BC0E6FF2CC0D8
:10220000E6FF5FEC21F02D6E050EE15E2D500D8A8C
:102210001D6A1E6A1F6A69D10101B92B400E0101B6
:10222000B95D02E10101B96B2D0E2A6E0101B951B0
:10223000EA6A400FE96E020EEA22EF502A5C28E1BA
:10224000040E2B6EFE0EDB502B5C22E0050E2C6E76
:10225000FE0EDB502C5C1CE0FE0EDB0406E0030EE1
:102260002A6EFE0EDB502A5C06E10D8C1D6A1E6A8A
:102270001F6A3BD10DD0010EF36E030EF3CFDBFFCF
:102280000101B92B400E0101B95D02E10101B96BF9
:10229000040E2A6EFE0EDB502A5C11E0050E2B6E3A
:1022A000FE0EDB502B5C0BE0050EE66ED9CFE6FF91
:1022B000DACFE6FF24D9E552E552E5523AD00101E2
:1022C000B951EA6A400FE96E020EEA22EFCF2AF016
:1022D0002B6A2C6A2AC0DFFF010E2BC0DBFF020E27
:1022E0002CC0DBFF050E2A6EFE0EDB502A5C19E1C6
:1022F000000EDBCFE6FF010EDBCFE6FF58EC22F04D
:10230000E552E552F3CF2AF0F4CF2BF02C6A2BBE26
:102310002C682AC0DFFF010E2BC0DBFF020E2CC091
:10232000DBFF0101B92B400E0101B95D02E10101A2
:10233000B96B030EDB5021E0DFCF2AF0010EDBCFBB
:102340002BF0020EDBCF2CF02268236824682AC011
:102350001DF02BC01EF02CC01FF033EC20F01AC073
:102360002AF01BC02BF01CC02CF02AC0DFFF010E8E
:102370002BC0DBFF020E2CC0DBFFFE0EDB5026E184
:10238000DFCF2AF0010EDBCF2BF0020EDBCF2CF0DB
:102390002C34000E2C1807E6D8807F0E2A54000E2D
:1023A0002B54000E2C5401E28CD0D9CFE9FFDACFA8
:1023B000EAFF020ED880EB50FF0A06E6800EEE5CC4
:1023C000FF0EEE58FF0EEF5801E27BD0FE0EDB044D
:1023D00024E1DFCF2DF0010EDBCF2EF0020EDBCF9C
:1023E0002FF02F34000E2F1807E6D880FF0E2D5443
:1023F000000E2E54000E2F5464E3D9CFE9FFDACF3C
:10240000EAFF020ED890EB50000A06E6000EEE5CE2
:10241000000EEE58000EEF5854E3020E306EFE0E22
:10242000DB50305C24E1DFCF31F0010EDBCF32F046
:10243000020EDBCF33F03334000E331807E6D880BA
:10244000FF0E31547F0E3254000E33543AE3D9CF8D
:10245000E9FFDACFEAFF020ED880EB50FF0A06E66A
:10246000000EEE5C800EEE58FF0EEF582AE3030ECE
:10247000346EFE0EDB50345C29E1DFCF35F0010E07
:10248000DBCF36F0020EDBCF37F03734000E3718D3
:1024900007E6D880FF0E3554FF0E3654000E375431
:1024A00010E3D9CFE9FFDACFEAFF020ED890EB5064
:1024B000000A06E6000EEE5C000EEE58000EEF5825
:1024C00005E20D8C1D6A1E6A1F6A0FD0DFCF2AF04D
:1024D000010EDBCF2BF0020EDBCF2CF02AC01DF05B
:1024E0002BC01EF02CC01FF000D0040EE15C02E2F5
:1024F000E16AE552E16EE552E7CFD9FF1200D9CF8C
:10250000E6FFE1CFD9FF020EE126FD0EDBCFE9FFAA
:10251000FE0EDBCFEAFFEE6AEE6AEE6A010EDB6AC0
:10252000FC0EDB50F36E010EDBCFF4FFF350F45CD6
:1025300055E20101B951EA6A400FE96E020EEA2242
:10254000EFCFDFFF300EDF5C44E3DF50390841E3BB
:10255000FD0EDBCFE9FFFE0EDBCFEAFFEECF2DF065
:10256000EECF2EF0EFCF2FF00A0E226E236A246AF0
:102570002DC01DF02EC01EF02FC01FF033EC20F038
:102580001AC02DF01BC02EF01CC02FF0300EDF5CE7
:10259000306E316A326A2D5030242A6E2E5031202E
:1025A0002B6E2F5032202C6EFD0EDBCFE9FFFE0E7E
:1025B000DBCFEAFF2AC0EEFF2BC0EEFF2CC0EEFF00
:1025C0000101B92B400E0101B95D02E10101B96BB6
:1025D00002D0000E05D0010EDB2AA2D7010E00D0DA
:1025E0002A6E020EE15C02E2E16AE552E16E2A50D7
:1025F000E552E7CFD9FF12000650E66EE66A1C0EE0
:102600002A6E3F0E2B6E2C6A2AC0E6FF2BC0E6FF17
:102610002CC0E6FF5FEC21F02D6E050EE15E2D5023
:1026200012000101D25108E0010E2A6E6D50020B1A
:1026300001E0010E2A5C22E10101D707000ED85B00
:102640000101D9510EE10101D751D81109E18B8067
:102650000101D00ED76F070ED86F0101010ED96F9F
:102660000CD00101D751D81108E18B900101D00E97
:10267000D76F070ED86F0101D96B5DD00101D2056C
:102680000CE0020E0101D25D08E0030E0101D25DF3
:1026900004E0050E0101D25D02E18B804CD0060EF4
:1026A0000101D25D48E10101D707000ED85B0101AD
:1026B000D9510EE10101D751D81109E18B800101F7
:1026C000100ED76F270ED86F0101010ED96F33D0CE
:1026D0000101D9050EE10101D751D81109E18B9013
:1026E0000101100ED76F270ED86F0101020ED96FAE
:1026F00022D0020E0101D95D0EE10101D751D8119E
:1027000009E18B800101A00ED76F860ED86F010101
:10271000030ED96F10D0030E0101D95D0CE3010146
:10272000D751D81108E18B900101100ED76F270EF9
:10273000D86F0101D96B120082B403D0010E03D00F
:1027400002D0000E00D01200E0EC18F0FB0EDBCF40
:10275000F3FFDB06F35000090AE02EEC19F0FA0E45
:1027600099EC19F0F3E12B1CF1E1010E01D0000E00
:102770000FEF19F0E0EC18F03B0EE12402E3E16802
:10278000E652E16E010EDB6A020EDB6AF90EDBCF68
:10279000F6FFFA0EDBCFF7FFFB0EDBCFF8FF0800EA
:1027A000F550DF6EDF5002E133EF18F0250EDF5CED
:1027B00002E026EF18F0030EDB6A040EDB6A050E5A
:1027C000DB6A060EDB6A070EDB6A48EC18F02D0E9A
:1027D000DF5C0CE02B0EDF5C09E0200EDF5C06E026
:1027E000230EDF5C03E0300EDF5C1AE1DF50300ABD
:1027F00014E0130A0FE0030A0AE00B0A05E0060AD8
:10280000E4E1030EDB80E1D7030EDB82DED7030EAB
:10281000DB84DBD7030EDB86D8D7030EDB88D5D766
:102820002A0EDF5C1BE144EC18F092EC18F010E08B
:10283000030EDB801E681F68130EDBCF23F0140E1F
:10284000DBCF24F07CEC20F0040E1CC0DBFF03D0B7
:10285000130E7BEC18F048EC18F00BD0090EDB6A75
:10286000E9EC18F003E05DEC19F0FAD7090E7BEC07
:1028700018F0030EDBB0DB982E0EDF5C1BE148EC9A
:1028800018F02A0EDF5C0BE144EC18F092EC18F023
:1028900003E1130ECDEC18F048EC18F00BD0090E44
:1028A000DB6AE9EC18F003E05DEC19F0FAD7090EE9
:1028B000CDEC18F0680EDF5C07E148EC18F0680E0C
:1028C000DF5C1DE1030E18D0740EDF5C17E07A0E9A
:1028D000DF5C14E0480EDF5C06E0540EDF5C03E0D2
:1028E0005A0EDF5C02E1020E07D06C0EDF5C03E0E3
:1028F0006A0EDF5C04E1010E20EC19F0C9DBDF5049
:102900006E0A01E17FD31E0A01E192D1200A01E1A2
:102910008FD13F0A01E149D11A0A01E146D10D0ADE
:1029200001E143D1200A01E140D13A0A01E13DD160
:10293000200A01E13AD1260A01E135D10D0A01E16F
:1029400032D11A0A01E1D9D0200A4AE0300A1FE048
:10295000460A0EE0250A01E083D3D950F90FE96E4B
:10296000FF0EDA20EA6E010EEE5E000EEE5AEE5A0F
:102970002EEC19F0250EE66E95DB03E12B1C01E130
:1029800069D32AEC19F001E26BD3DB2A69D3080E74
:10299000DB6A040EDB50010806E2040EDB04F2ECF5
:1029A00018F0DB508BDB080EDB5009E0030EDB5028
:1029B000010B05E172DB01E04DD3080EDB6A64DB3D
:1029C000EFCFDFFFA2EC19F003E12B1C01E142D3B2
:1029D0002AEC19F001E3DB2A60DB01E141D33AD3B1
:1029E000070EDB5002080FE16EEC19F0030E35EC18
:1029F00019F00E0EEECFDBFF0F0EEECFDBFF100E49
:102A0000EECFDBFF20D0F70EDBCF2DF0F80EDBCFC3
:102A10002EF0020E2D5E000E2E5AF70E2DC0DBFF9B
:102A2000F80E2EC0DBFF2DC0E9FF2EC0EAFF25EC1B
:102A300019F02C6A0E0E2AC0DBFF0F0E2BC0DBFF35
:102A4000100E2CC0DBFF0E0EDBCFE6FF0F0EDBCF30
:102A5000E6FF100EDBCFE6FF33EC22F0E552E55245
:102A6000E552130E1DC0DBFF140E1EC0DBFF060E69
:102A7000DB5005E0130E69EC19F001E26ADB8DEC26
:102A800019F002E2130E37DB50EC19F006E0040EE9
:102A900069EC19F002E2050E2EDB030EDBB005D067
:102AA000FCDA01E0D7D2080EDB6A090EDB6A0E0EF3
:102AB000DBCFF6FF0F0EDBCFF7FF100EDBCFF8FFFB
:102AC0000800F550DF6EDF5014E093EC19F011E2CE
:102AD000A2EC19F003E12B1C01E1BCD2BBDB01E34A
:102AE000DB2A090EDB2AD9500E0FE96E000ECBDB74
:102AF000E7D7D3DA01E1B4D2ADD2C6DA110EEECF08
:102B0000DBFF120EEDCFDBFF110EDBCFE6FF120E67
:102B1000DBCFE6FF25EC22F0E552E552130EF3CFB2
:102B2000DBFF140EF4CFDBFF060EDB5004E0130EC8
:102B3000D0DB01E20EDB8DEC19F002E2130EDBDAE2
:102B4000AFDB05E0040EC5DB02E2050ED4DA030EAE
:102B5000DBB005D0A2DA01E07DD2080EDB6A090EF7
:102B6000DB6A110EDBCFE9FF120EDBCFEAFFEFCFFE
:102B7000DFFFDF5014E0D7DB12E2E4DB03E12B1CC4
:102B800001E168D267DB01E3DB2A090EDB2A110EC3
:102B9000DB2ADBCFE9FF120EE8E3DB2AE6D77DDA9A
:102BA00001E15ED257D2030EDB8E070EDB0410E18B
:102BB00095DB040E5ADB0A0EEECFDBFF0B0EEECFD9
:102BC000DBFF0C0EEECFDBFF0D0EEECFDBFF6CD08C
:102BD000070EDB5003082CE1030EDBAE0DD0B2DA9A
:102BE000020E76DAEFCF2AF02B6A2C6A2D6A2AAE13
:102BF00039D02B682C6835D0F70EDBCF2BF0F80ED0
:102C0000DBCF2CF0020E2B5E000E2C5AF70E2BC0E1
:102C1000DBFFF80E2CC0DBFF2BC0E9FF2CC0EAFF66
:102C2000EFCF2AF00A0E2AC0DBFF0B0EDB6A38D08A
:102C3000070EDB50020809E1030EDBAE04D059DBBE
:102C40002CAE10D00ED055DB0DD0030EDBAE12D063
:102C500079DA020E3DDAF9DA2C6A2D6A2BAE02D04F
:102C60002C682D68E2DA0C0E2CC0DBFF0D0E2DC097
:102C7000DBFF1AD0F70EDBCF2CF0F80EDBCF2DF0F8
:102C8000020E2C5E000E2D5AF70E2CC0DBFFF80E44
:102C90002DC0DBFF2CC0E9FF2DC0EAFFD6DAC5DA74
:102CA0000C0EDB6A0D0EDB6A060EDB5005E1010E31
:102CB000F36E050EF3CFDBFF150EDB6A160EDB6A33
:102CC000D950370F2A6E000EDA202B6E390E2AC02B
:102CD000DBFF3A0E2BC0DBFF380EDB6A080EDB6A27
:102CE0000A0EAEDADF50780A12E0200A10E0280A55
:102CF0000CE0200A0AE03F0A06E00D0A02E0200A82
:102D000008E1020E05D0080E03D0080EDF26100ED3
:102D100097DA030EDBBE02D0DB92DB94DB50800B34
:102D200024E08ADAD890030EEB50000A08E6000E81
:102D3000EE5C000EEE58000EEE58000EEE5815E256
:102D400013DA2168226823682468EDEC21F00A0E6A
:102D500018C0DBFF0B0E19C0DBFF0C0E1AC0DBFF27
:102D60000D0E1BC0DBFF2D0E08D0030EDBA202D020
:102D70002B0E03D0DBA408D0200EF36E170EF3CF7A
:102D8000DBFF150EDB2A02D0170EDB6A050EDB50C7
:102D900003E1B7D901E189D0E80E2A6E450E2B6E0A
:102DA000000E2C6E070EDBCF2DF02E6A2F6A306AD4
:102DB0002DC021F02EC022F02FC023F030C024F00F
:102DC000D3D97EEC22F02A501824F36E2B50192010
:102DD000F46E2C501A20F86EF4CFF7FFF3CFF6FF05
:102DE0000800090EF5CFDBFF580EDF5C0FE1610E26
:102DF000F36E090E7BD90AE3200E2A6E090EDBCF93
:102E0000E7FF2A50E75E090EE7CFDBFF070EDBCFB7
:102E10002AF02B6A2C6A2D6A0FDA2AC021F02BC007
:102E200022F02CC023F02DC024F0EECF1CF0EECF0A
:102E30001DF0EECF1EF0EFCF1FF07EEC22F01FC092
:102E4000EDFF1EC0EDFF1DC0EDFF1CC0EFFF390EF2
:102E5000DBCFE9FFDB063A0EDBCFEAFF01E2DB0660
:102E6000090EDBCFEFFF150EDB2A4BD995E1030EE0
:102E7000DBA61DD06F0EDF5C06E1C1D918E3150E8D
:102E8000DB285BDA14D0780EDF5C09E0580EDF5CDB
:102E900006E0620EDF5C03E0420EDF5C08E1020E3A
:102EA000F36E160EF3CFDBFF02D0150EDB6A030EB6
:102EB000DB50100B0EE0040EDBCF2AF0050EDB50CA
:102EC000D8802A5406E2060EDB5003E1040EDB50E4
:102ED00034DA95D90AE2050EDBCFE7FF150EDB5099
:102EE000E75E050EE7CFDBFF02D0050EDB6A040EBE
:102EF000DBCF2AF0160E45D9D8802A5414E2160EDC
:102F0000DBCFE6FF150EDBCFE6FF040EDBCFE6FFDF
:102F1000050EDB50E552E75CE552D880E754E552F8
:102F2000D880E7545FD9030EDB50010B0BE1080E8C
:102F3000DB5008E0B2D801E08DD0080EDB50BED8DF
:102F4000080EDB6A170EDB5007E088D9170EF1D99F
:102F500003E12B1C01E17ED0160EDB5016E07ED97A
:102F6000300EE66E9FD802E12B1C74E077D9DFCFDC
:102F7000E6FFABEC21F0E552E552E552F4CF2BF041
:102F80000001F31C02E12B1C65E0050EDBCF2AF0EB
:102F9000160EDB50D8802A5409E2050EDBCFE7FF7E
:102FA000160EDB50E75E050EE7CFDBFF300EE66E58
:102FB000050ECBD94FE1390EDB2ADBCFE9FF3A0E04
:102FC00001E3DB2ADBCFEAFF090EEFCFDBFFDB50AB
:102FD0000EE044D9090EADD902E12B1C3BE0390EBD
:102FE000DB2ADBCFE9FF3A0EEDE3DB2AEBD755D83E
:102FF00031E1160EDBCFE6FF080EC3D8E552E72419
:103000005DD82ED0070EDB50030A1CE0010A14E045
:10301000030A07E07BD9DBCFEEFF020EDBCFEDFF2B
:103020001FD0F5D82F6A2DAE02D02E682F682CD86D
:10303000BCD82FC0EEFF14D0EAD82DBE2E6824D8FD
:10304000B4D80ED063D9DBCFEFFF0AD07BD905E12E
:103050002B1C03E1F368F46810D0FCD801E3DB2AF1
:1030600079D9CFEF13F0010EDBCF2AF0020EDBCFC0
:103070002BF02AC0F3FF2BC0F4FF3B0EE15C02E211
:10308000E16AE552E16ECBD029D9020E35EF19F095
:1030900061D90800F550DF6E1200200EE66E080EB2
:1030A000A5EF19F0ABEC21F0E552E552E552F3CF74
:1030B0002AF0F4CF2BF00001F31C12002A6E2B6AC9
:1030C000D950010F4DD92A50EE262B50ED22120077
:1030D0002E5E000E2F5AF70E2EC0DBFFF80E2FC00B
:1030E000DBFF2EC0E9FF2FC0EAFF1200DBCFF4FFA9
:1030F000F350F45C1200DB50E76E040EE7CFDBFF09
:1031000012000A0EDBCF2AF00B0EDBCF2BF00C0ED9
:10311000DBCF2CF00D0EDBCF2DF02A502B102C1016
:103120002D101200130EEECFDBFF140EEDCFDBFFE0
:10313000130EDBCF2AF0140EDBCF2BF00001800E34
:103140002B141200F70EDBCF2EF0F80EDBCF2FF092
:103150001200050EDB50E66ED950130F01D9E5526F
:10316000E750EE6EED6A12000A0EDBCF1CF00B0E7C
:10317000DBCF1DF00C0EDBCF1EF00D0EDBCF1FF0F2
:103180001200DBCFE6FF150EDBCFE6FF050EDB50AE
:10319000E552E724E552E7241200DB50CED8010EB9
:1031A000F36E060EF3CFDBFF1200EE50EFCFEAFF17
:1031B000E96E2CC0EEFF2DC0EEFF2EC0EEFF120018
:1031C000D9CFE6FFDACFE6FFE1CFD9FFE2CFDAFFD2
:1031D0001200DFCFE6FFE66A6CEC22F0E552E55222
:1031E000F3501200E76E080EE7CFDBFF1200EECFC0
:1031F0002AF0EECF2BF0EFCF2CF02D6A1200050E47
:10320000DBCF2AF0150EDB50D8802A541200010EB5
:10321000DBCF2CF0020EDBCF2DF02E6A1200E55230
:10322000E5CFDAFFE7CFD9FF12000A0E2AC0DBFF95
:103230000B0E2BC0DBFF1200D9500A0FB0EF19F0B4
:10324000F36E070EF3CFDBFF1200EECF2AF0EFCFC5
:103250002BF01200010EDB2A020E1200FC0EDBCF57
:10326000E6FFFD0EDBCFE6FF12002A5E000E2B5AB2
:10327000F70E2AC0DBFFF80E2BC0DBFF2AC0E9FFE8
:103280002BC0EAFF1200DA20EA6EEF2AEECFF6FF3B
:10329000000EEF22EECFF7FFEF22EECFF8FF120085
:1032A000040EDBCFE6FF130EDB50E552E75C9ADF3E
:1032B000DB5004DF060EDB501200090EDB500A0D56
:1032C000F350DF24D00FE76E090EE7CFDBFF48EFA6
:1032D00018F0DB50F36E050E76EF18F0F70EDBCF2B
:1032E0002AF0F80EDBCF2BF01200DFCFE6FF52EF13
:1032F00018F028DF030EECDEF7EF18F0A4EC13F063
:10330000E552E552E552E55200091200BDDEEE50ED
:10331000EFCFEAFFE96E010E1200130EDB50F36EE1
:10332000040E76EF18F0040EDB50F36E090E76EF04
:1033300018F0DBCFE6FF52EF18F0E76E050EE7CF8F
:10334000DBFF12008BDF75EF19F0DBCFE6FF86DFC6
:103350007EEF19F0D950F90FE96EFF0E43EF19F027
:10336000E96E000EDA20EA6E1200040120511F0BF4
:10337000010801E060D004012051600BE842E842FE
:10338000E842E842E842010801E055D00401245136
:1033900004E00401240501E04ED004012151230A78
:1033A00048E0010A40E0030A30E0010A25E0240A6F
:1033B00022E0070A1FE0010A1CE0030A11E0010AEB
:1033C00001E038D00101030ECB6F0101A90ECC6FD3
:1033D000010ECD6F0101D3930101080ED06F2BD0E8
:1033E0000101030ECB6F0101A90ECE6F010ECF6F4D
:1033F00022D021D020D01FD00101030ECB6F0101BC
:10340000A10ECE6F010ECF6F16D00101030ECB6F50
:103410000101A10ECC6F010ECD6F0101D39301010B
:10342000070ED06F08D00101030ECB6F22C4A8F1A4
:1034300002D001D000D012000101A16BC20EA26F18
:10344000010EA36FA46B0101A56B0101A66B010125
:10345000080EA76F01019A6B0101996B1A0E726E2B
:103460001E0E736E0401000E166F050E176F040119
:10347000400E146F0401400E196F0401080E1A6FFC
:10348000050E1B6F0401880E186F0401480E1E6F95
:10349000050E1F6F0401400E1C6F1200D9CFE6FF0E
:1034A000E1CFD9FF0101996B040118BF39D0FC0E9F
:1034B000DBCF2AF004011951D8802A5403E2FC0E14
:1034C00019C4DBFF0101996BFC0EDB500101995D12
:1034D0001CE201019951EA6A080FE96E050EEA2221
:1034E000EF50E66E01019951E76EFD0EDBCFE9FF6B
:1034F000FE0EDBCFEAFFE750E926000EEA22E55296
:10350000E750EF6E0101992BDFD70401400E196FD0
:10351000400E040118170401187D880E04011813C9
:103520000101995100D0E552E7CFD9FF1200D9CF60
:10353000E6FFE1CFD9FFE65201019A5101E031D017
:10354000DF6ADF2ADF502A6E2B6A2A5002E1010E61
:103550002B1801E10BD0FD0EDBCFE9FFDB2AFE0EBD
:10356000DBCFEAFF01E3DB2AEF50EBE1DF502A6E0D
:103570002B6AD950FD0FE96EFF0EDA20EA6E2A5051
:10358000EE5E2B50ED5ADF06FD0EDBCF9BF1FE0EFB
:10359000DBCF9CF1DFCF9FF10101A06B0101010E98
:1035A0009A6FE552E552E7CFD9FF1200D9CFE6FF77
:1035B000E1CFD9FFE65201019A5101E033D0DF6A31
:1035C000DF2ADF502A6E2B6AFF0E2A1801E12B50EA
:1035D00001E10CD0FD0EDBCFF6FFDB2AFE0EDBCFC8
:1035E000F7FF01E3DB2A0800F550EAE1DF502A6E1D
:1035F0002B6AD950FD0FE96EFF0EDA20EA6E2A50D1
:10360000EE5E2B50ED5ADF06FD0EDBCF9BF1FE0E7A
:10361000DBCF9CF1DFCF9FF10101010EA06F010113
:10362000010E9A6FE552E552E7CFD9FF1200D9CFCC
:10363000E6FFE1CFD9FFE65204011CBF7DD0030EA7
:1036400001019A5D02E101019A6B01019A5101E1C8
:1036500073D0020E01019A5D06E104011D6B0101A8
:10366000030E9A6F61D001019A055EE1400E2A6E49
:103670002B6A01019F512A5C000E2B5803E2400E79
:10368000DF6E02D09FC1DFFFDFCF1DF4DF500101ED
:103690009F5D01019F6F0101480E9D6F050E9E6F9A
:1036A0000101A00518E1DF5015E09BC1F6FF9CC1A8
:1036B000F7FF0800F5509DC1E9FF9EC1EAFFEF6EDC
:1036C00001019D2B000E9E2301019B2B000E9C23CC
:1036D000DF06E9D716D0DF5014E09BC1E9FF9CC19B
:1036E000EAFFEF509DC1E9FF9EC1EAFFEF6E0101C5
:1036F0009D2B000E9E2301019B2B000E9C23DF06B9
:10370000EAD701019F5110E104011D512A6E2B6A75
:10371000400E2A1801E12B5004E10101020E9A6FBC
:1037200003D00101030E9A6F400E04011C1704011F
:103730001C7D880E04011C13E552E552E7CFD9FF2A
:1037400012006C5002E0000E01D0010E00090BE0E7
:10375000040100513C0BE842E8420D0802E10CD89C
:1037600001D042D808D06C5002E0000E01D0010E0A
:10377000040901E04BD81200D9CFE6FFE1CFD9FF11
:10378000E6520101CA6B0101CB6B0101D06BD16B19
:103790003EEC1DF0DF6ADF502A6E2B6A010E2A5CB8
:1037A000000E2B581BE20101CB5101E017D0F76A44
:1037B000DF34FE0BF736F66E1D0EF626420EF722AC
:1037C0000900F5CF2AF00800F5CF2BF004D02BC06C
:1037D000FAFF2A50F96EFBDFDF2ADDD7F0D8E55279
:1037E000E552E7CFD9FF1200020E0101CA5D0CE1DC
:1037F000A4D8040100BD04D00401C80E006F03D09A
:103800000401880E006F01D029D91200040E0101B5
:10381000D25D0CE122C46EFF6E50000804E201018B
:10382000050ED26F03D00101030ED26F0101CA054C
:103830000CE10DD8040104BD04D00401C80E046FCE
:1038400003D00401880E046F01D008D91200D9CF2B
:10385000E6FFE1CFD9FF020EE1260101080ED05D9F
:10386000000ED15905E2D0C1DEFFD1C1DDFF03D08A
:10387000080EDE6EDD6A0401049304010491010E5A
:10388000DB5004010413DFCF05F4000EDB5001010F
:10389000D05F010EDB500101D15B0101280ECE6F1C
:1038A000040ECF6F0101D3A320D0D9CFE9FFDACF27
:1038B000EAFFEE50ED1018E0CCC1F6FFCDC1F7FFE6
:1038C0000800F550CEC1E9FFCFC1EAFFEF6E01015C
:1038D000CE2B000ECF230101CC2B000ECD23DF0613
:1038E000010E01E2DB06E1D71ED0D9CFE9FFDACF26
:1038F000EAFFEE50ED1017E0CCC1E9FFCDC1EAFFC1
:10390000EF50CEC1E9FFCFC1EAFFEF6E0101CE2B30
:10391000000ECF230101CC2B000ECD23DF06010EBC
:1039200001E2DB06E2D7020EE15C02E2E16AE55267
:10393000E16EE552E7CFD9FF1200D9CFE6FFE1CF24
:10394000D9FF020EE126030E04010015E76E010EF9
:10395000E7CFDBFF01C4DFFFDE500101D027DD50E0
:103960000101D1230101280ECC6F040ECD6FD9CFF8
:10397000E9FFDACFEAFFEE50ED1017E0CCC1E9FF26
:10398000CDC1EAFFEF50CEC1E9FFCFC1EAFFEF6E34
:103990000101CE2B000ECF230101CC2B000ECD2335
:1039A000DF06010E01E2DB06E2D7020EE15C02E275
:1039B000E16AE552E16EE552E7CFD9FF12006D985A
:1039C0000101CB510FE10401080E016F0401200E2B
:1039D000026F040E036F0401840E006F0401840E55
:1039E000046F3BD0040120AF25D00101D051040168
:1039F000265D0101D1510401275904E226C4D0F10A
:103A000027C4D1F124DF0101010ECA6F0401080EA1
:103A1000016F0401200E026F040E036F0401800E7B
:103A2000006F0401280E066F040E076F0401C80E14
:103A3000046F13D00101020ECA6F0401056B04016B
:103A4000C80E046F0401080E016F0401280E026FF6
:103A5000040E036F0401C80E006F12000101CA6B4F
:103A60000401080E016F0401200E026F040E036FA3
:103A70000401880E006F0401046B12000401205140
:103A8000600BE842E842E842E842E842000901E00F
:103A900058D004012151070A53E00B0A51E0070AEC
:103AA00042E0010A2CE00B0A28E0020A26E0030AA1
:103AB00022E0080A12E0010A0EE00F0A0AE0030AF7
:103AC00001E03ED00101010ECB6F0101040ED26F67
:103AD00038D038D836D093D834D00101010ECB6F0E
:103AE0000101D40ECC6F010ECD6F0101D393010102
:103AF000010ED06F26D0ABD824D0F9D822D0010146
:103B0000010ECB6F040124510101CC6FCD6BD50E9A
:103B10000101CC27010E0101CD230101D393010145
:103B2000010ED06F0ED00101010ECB6F04012451A4
:103B3000EA6AD50FE96E010EEA2222C4EFFF01D036
:103B400000D01200800E0401205D58E104012351D1
:103B5000030A34E0010A10E0030A01E04DD001013C
:103B6000010ECB6F0101520ECC6F410ECD6F120EC4
:103B70000101D06FD16B40D00101010ECB6F040168
:103B80002251F66EF76AD890F636F736130EF626FF
:103B9000420EF7220900F5CFCCF10A00F5CFCDF1A6
:103BA000020E0101F76ACC25F66ECD51F72209000D
:103BB000F5CFD0F10A00F5CFD1F11ED00101010EF1
:103BC000CB6F04012251F66EF76AD890F636F736BD
:103BD000170EF626420EF7220900F5CFCCF10A00A7
:103BE000F5CFCDF1CCC1F6FFCDC1F7FF0800F55000
:103BF0000101D06FD16B00D00101D383120001010C
:103C0000010ECB6F0F0EE66E710EE66E0F0EE66EB6
:103C100079EC1FF0E552E552E552010EE66ED50E45
:103C2000E66E010EE66E79EC1FF0E552E552E552C4
:103C300022C4D4F10401225104E10101050ED26F26
:103C400005D00101060ED26F1CEC1AF0120004011F
:103C5000286B0401296B040120511F0B020A14E098
:103C6000030A0EE0010A01E034D00101010ECB6F1E
:103C7000040128810101D3A102D00401288329D0A5
:103C80000101010ECB6F25D00101010ECB6F0401A4
:103C900024510F0B080DF3502B6A000F2A6E040EEF
:103CA0002B2204012451800B01E0010E040DF3507E
:103CB00001012A24CE6F000E2B20CF6FCEC1E9FF69
:103CC000CFC1EAFFEF50040B03E00401010E286F9F
:103CD00000D00101CB050AE10101280ECC6F040ED2
:103CE000CD6F0101D3930101020ED06F12000401C8
:103CF000220511E1040120511F0B00090CE1010113
:103D0000010ECB6F030E0401215D03E10101D3819C
:103D100002D00101D391040122513EE1040120515E
:103D20001F0B020839E1040124510F0B000934E094
:103D30000101010ECB6F040124510F0B080DF3504C
:103D40002B6A000F2A6E040E2B2204012451800BD3
:103D500001E0010E040DF35001012A24CE6F000E84
:103D60002B20CF6F030E0401215D07E1840ECEC12D
:103D7000E9FFCFC1EAFFEF6E0FD0040124AF06D0F8
:103D8000CEC1E9FFCFC1EAFFEF6A06D0880ECEC1EF
:103D9000E9FFCFC1EAFFEF6E12006DA610D802D086
:103DA0006DB614D80101D20509E16DBA07D0686A71
:103DB000696A698069880101020ED26F12006D6A1A
:103DC000696A6D860101010ED26F12006D6A696A1F
:103DD0000101D26B1200FADF12000101D25101E1A0
:103DE0003AD06850040B04E06950040B01E03CD861
:103DF0006DB231D06850010B04E06950010B01E055
:103E000056D86850100B04E06950100B01E024D81C
:103E10006850400B04E06950400B01E03DD8685009
:103E2000200B04E06950200B01E038D86850020BE9
:103E300004E06950020B01E038D8030E0101D25DA5
:103E400001E209D06850080B06E06950080B03E056
:103E5000A1EC1BF068961200698468986D82A19AA3
:103E6000A08A0300A09A12006D92699468941200CF
:103E70000101D3A110D0F8DF6D840101080EDA6FC3
:103E8000070EDB6F0101DA07000EDB5B0101DA517F
:103E9000DB11F8E16D941200689C120070A003D051
:103EA0002EEC1DF07090689A1200689212006A6AF7
:103EB000686A9F0E6B6E7B0E696E6E6A0F0EE66E01
:103EC000710EE66E0F0EE66E14D8E552E552E5521D
:103ED000160E706E68A602D06896FCD76D982EEC10
:103EE0001DF00101D3910101D46B0101030ED26FCA
:103EF0001200D9CFE6FFE1CFD9FFFD0EDBCFE9FFFE
:103F0000FE0EDBCFEAFFFC0EDB5004E0EE6AFC0E97
:103F1000DB06F9D7E552E7CFD9FF1200537461747D
:103F200075733D25690D0A002135204572723A20CE
:103F30004E65656420636F6D6D61206E6578742CCD
:103F400020666F756E643A20272563270D0A00509E
:103F5000492C2531750D0A004D522C253033750D35
:103F60000A002C25303475004100492C2530336976
:103F70002C253033692C253033690D0A0021382077
:103F80004572723A20556E6B6E6F776E20636F6D5F
:103F90006D616E642027256325633A2532582532EA
:103FA00058270D0A002138204572723A20556E6B51
:103FB0006E6F776E20636F6D6D616E642027256371
:103FC0003A253258270D0A002137204572723A20CF
:103FD0004578747261207061726D617465720D0A4A
:103FE000002136204572723A20496E76616C696410
:103FF00020706172616D7465722076616C75650DFB
:104000000A002134204572723A204D697373696E3B
:104010006720706172616D657465722873290D0A7D
:10402000002133204572723A20525820427566664C
:104030006572206F76657272756E0D0A00213220EE
:104040004572723A20545820427566666572206F38
:1040500076657272756E0D0A002131200D0A0021FD
:1040600030200D0A00FF1FC029F01EC028F01DC01F
:1040700027F01D502202F4CF1BF0F3CF1AF01E5090
:104080002302F4CF1DF0F3CF1CF02202F3501B26C5
:10409000F4501C22E86A1D2227502302F3501B26ED
:1040A000F4501C22E86A1D221F502202F3501C26E5
:1040B000F4501D221F5023021E6AE86A1E22F3508C
:1040C0001D26F4501E2227502402F3501C26F450C3
:1040D0001D221F6AE86A1E221F2228502402F35064
:1040E0001D26F4501E22E86A1F2229502402F35094
:1040F0001E26F4501F22000C1FC029F01EC028F0FD
:104100001E502302F4CF1DF0F3CF1CF01F502402E9
:10411000F4CF1FF0F3CF1EF02302F3501D26F4500E
:104120001E22E86A1F2228502402F3501D26F45054
:104130001E22E86A1F2224AEA2EF20F028501E5E45
:1041400029501F5A29AE000C23501E5E24501F5ABE
:10415000000C1201000202000008D8040A0000004E
:10416000010200010902430002010080320904003B
:1041700000010202010005240010010424020205CE
:10418000240600010524010001070582030800023E
:1041900009040100020A00000007050302400000B4
:1041A000070583024000000403090434034D00693D
:1041B00000630072006F00630068006900700020F7
:1041C0000054006500630068006E006F006C006FB3
:1041D0000067007900200049006E0063002E003463
:1041E000034300440043002000520053002D0032DE
:1041F0000033003200200045006D0075006C006146
:1042000000740069006F006E002000440065006DBE
:10421000006F0064416441A741AB41DF416A33FF55
:104220002A0EF66E080EF76E000EF86E01010900F8
:10423000F550C56F0900F550C66F03E1C56701D0A1
:104240003DD00900F550C06F0900F550C16F09005D
:10425000F550C26F09000900F550E96E0900F550EC
:10426000EA6E090009000900F550C36F0900F55016
:10427000C46F09000900F6CFC7F1F7CFC8F1F8CF36
:10428000C9F1C0C1F6FFC1C1F7FFC2C1F8FF01010A
:10429000C35302E1C45307E00900F550EE6EC307B3
:1042A000F8E2C407F9D7C7C1F6FFC8C1F7FFC9C113
:1042B000F8FF0101C507000EC65BBFD71200D9CFBA
:1042C000E6FFDACFE6FFE1CFD9FFE2CFDAFFE65231
:1042D000E652E652E652D950FB0F2A6EFF0EDA2064
:1042E0002B6E2AC0DEFFDD6EDECFE6FFDDCFE6FF00
:1042F000FB0EDBCFE6FFFC0EDBCFE6FFFD0EDBCFD8
:10430000E6FFDCC1E6FFDDC1E6FFBAEC13F02A6E82
:10431000070EE15C02E2E16AE552E16E2A50020E0C
:10432000F3CFDBFF030EF4CFDBFF020EDBCF2AF06F
:10433000030EDBCF2BF02AC0F3FF2BC0F4FF040EDB
:10434000E15C02E2E16AE552E16EE552E5CFDAFFB7
:10435000E7CFD9FF1200D9CFE6FFDACFE6FFE1CFF2
:10436000D9FFE2CFDAFFFB0EDBCF2AF0FC0EDBCF6A
:104370002BF00001800E2B141AE1FB0EDBCFE9FFBE
:10438000FC0EDBCFEAFFEECFF3FFEDCFF4FFEE2A1A
:10439000000EEF22F3CFE9FFF4CFEAFFFD0EDBCFF3
:1043A000EFFFEF502B6AF36E2BC0F4FF10D0FB0E23
:1043B000DB50FE0806E1FD0EDBCFE6FFCFEC22F07E
:1043C00005D0FD0EDBCFE6FFB3EC07F0E552E5527A
:1043D000E5CFDAFFE7CFD9FF12001C502102F3CF5F
:1043E00018F0F4CF19F02202F3501926000EF42031
:1043F0001A6E1C502302F3501A26000EF4201B6E76
:104400001C502402F3501B261D502102F350192684
:10441000F4501A22000E1B221D502202F3501A26BD
:10442000F4501B221D502302F3501B261E50210264
:10443000F3501A26F4501B221E502202F3501B2662
:104440001F502102F3501B261200FE0EE3CFE9FF9E
:10445000FF0EE3CFEAFFF36AF46AEE5203E0F34A99
:10446000F42AFBD71200FF0EE3CFF8FFE552FF0E50
:10447000E3CFF7FFE552FF0EE3CFF6FFE552E66A22
:10448000E66AE66A0900F55209E0FD0EE32A05E155
:10449000FE0EE32A02E1FF0EE32AF4D7FD0EE3CF7E
:1044A0001DF0FE0EE3CF1EF0FF0EE3CF1FF0120053
:1044B000FF0EE124E96EFF0EE220EA6EEDCFF4FF7D
:1044C000EFCFF3FFF46607D0600EF36404D07B0EE9
:1044D000F36001D0F39A1200F36AF46AFF0EE1244C
:1044E000E96EFF0EE220EA6EED6607D02F0EEF6454
:1044F00004D03A0EEF6001D0F32A12001B6A1A6A48
:10450000196A186A200EE76ED8901C361D361E36C2
:104510001F36183619361A361B362150185C2250B1
:10452000195823501A5824501B5809E32150185E7B
:104530002250195A23501A5A24501B5A1C2AE72E6B
:10454000E4D7120005D811D88FEC06F0FCD7120082
:104550000F0EC112140E6F6E0101D26B0101D36BED
:104560000101D46BC4EC05F01200CDEC1EF06FBE5F
:1045700002D0EDEC1EF017EC1BF012004F4B0D0AB1
:10458000000D0A00554257204657204420566572B8
:1045900073696F6E20312E342E330D0A00FFFF0E2B
:1045A000E350ACBA04D0AF6AAB8EAC8A949CACA298
:1045B000FED7AD6EF36EF46A120013EE00F023EE38
:1045C00000F0F86A179C10EC21F0A2EC22F0FDD765
:1045D0001200FF0EE350E84E1200000000D000D0A1
:1045E00000D0E82EFAD71200303132333435363766
:1045F000383961626364656600FF00EE00F00F0EFB
:10460000EE6AEA62FDD7120000000000FEFFFFFF25
:10461000FFFFFFFFFFFFFFFFFFFFFFFFFFFFFFFFAA
:10462000FFFFFFFFFFFFFFFFFFFFFFFFFFFFFFFF9A
:10463000FFFFFFFFFFFFFFFFFFFFFFFFFFFFFFFF8A
:10464000FFFFFFFFFFFFFFFFFFFFFFFFFFFFFFFF7A
:020000040030CA
:0E000000250E3A1E008181000F800FA00F40D8
:00000001FF
